:1000000000A8000000050000A1680000000000003A
:1000100000000000000000000000000000000000E0
:10002000801878FFE4B8200118F6D8F99000007F16
:10003000007E07E4F0A3DFFCDEFA75812102328E38
:10004000EFB4100575B2928007EFB4040B75B28E51
:1000500075B6F9E4F5B7800DEFB4080975B28E7581
:10006000B6F375B70143B20122320002297A7F0547
:10007000123AB21238EE1233CA9002367401F0020C
:100080002F76000235F475B28E75B6F9E4F5B743F4
:10009000B20143AA01023A9900000002104925E08A
:1000A00025E0241CF582E43403F583E0F8A3E0F9AD
:1000B000A3E0FAA3E0FB900328E0FCA3E0FDA3E0AB
:1000C000FEA3E02275F00212229175F099E0FCA3E4
:1000D000E0FDEFA42451F582E5F03400F58322EF32
:1000E0002466FFEE34FEFE7C007D0A12217A7D320A
:1000F00012218CEF249AFFEE3401FEEB75F002A47E
:100100002433F582E5F03400F5832275F0021222E3
:100110009175F099E0FCA3E0FDEFA42463F582E57E
:10012000F03400F58322901F2EC39BFBEE9AFAED6C
:1001300099F9EC98F8E493FE740193FFE4FCFDC395
:1001400002224375F099EEA424B4F582E5F0340060
:10015000F583E5822FF582E43583F583E4F075F0CD
:1001600099EEA424BDF582E5F03400F583E5822FF5
:10017000F582E43583F58322E0FEA3E0FF9003E4FB
:10018000E0FD75F002A42487F582E5F03400F583E4
:10019000EE8FF012221775F002EDA42487F582E5A8
:1001A000F03400F58322EF2424FFEE34FAFE7C00C5
:1001B0007D0A12217A7D1E12218CEF24DCFFEE34A1
:1001C00005FEEB75F002A4242DF582E5F03400F570
:1001D00083229003D0E0FE75F099A4243FF582E5D8
:1001E000F03400F583EF75F002022291F583E49379
:1001F000FC740193FD75F002EFA42410F582E5F084
:100200003402F583ECF0A3EDF09003D1E02275F019
:1002100002EBA42427F582E5F03400F583E0FCA38B
:10022000E0FDEB75F002A42421F582E5F03400F541
:1002300083229003D1E075F099A42475F582E5F04E
:100240003400F58322F583E493FC740193FD75F08B
:1002500002EFA4229003E4E0FD75F099A42499F53F
:1002600082E5F03400F5832275F099EFA4243FF580
:1002700082E5F03400F583EE75F002022291C39B13
:10028000FBEE9AFAED99F9EC98F822E04401F0E4DB
:10029000900020F0900316229003E475F099E0FF9F
:1002A000A4243FF582E5F03400F58322F0A3F0A307
:1002B000F0A3F0A3F0A3F0A32275F002EBA424278F
:1002C000F582E5F03400F5832275F002EC122291FC
:1002D000E0FEA3E0FFD3229003D1E025E024D3F594
:1002E00082E43403F58322C3E0FDEF9D7480F86E51
:1002F000982275F002A4240AF582E5F0340222E087
:10030000241CF582E43402F58322E0FEA3E0C39DC1
:10031000FFEE9C229003E4E0FF75F09922F583E064
:10032000FCA3E0FD75F00222F0900346E054F0F0EB
:1003300022FFEB25E025E022F583E4F07F0122CBCC
:10034000EFCBEBD394032275F002A42416F582E5DB
:10035000F03402229003E4E0FF241FF582E434022B
:10036000F5832274222EF582E43402F58322900371
:10037000ECE0FF24B4F582E43400F58322E0FCA332
:10038000E0FD75F09922ECF0A3EDF09003E5E004B8
:10039000F022E04406F09000207401F0229003E780
:1003A000E0FEA3E0FF9003E4E0FD75F09922EE8FFC
:1003B000F012221775F09922EB25E024E0F582E493
:1003C0003420F58322EF25E024D9F582E43403F5C7
:1003D000832290001FE0FF9003D1E0C39F22E4F04E
:1003E000A3F075F0992274972BF582E43402F5831B
:1003F0002274492BF582E43402F5832274F02BF544
:1004000082E43402F58322742E2BF582E43403F562
:10041000832274072BF582E43403F5832274382B8E
:10042000F582E43402F5832274032BF582E4340070
:10043000F5832274582BF582E43402F58322741775
:100440002BF582E43403F58322742E2EF582E434F6
:1004500002F5832275F099A424B4F582E5F0340006
:10046000222401FFE43EFEE43DFDE43CFC90032831
:10047000022254E0FCA3E0FDEC541F22F0A3F0A301
:10048000F0A3F0A322E4F0A3F075F00222F074BD13
:100490002FF582E43400F5832290022DE0640122DE
:1004A000E49003C6F09002367402F022E490022633
:1004B000F0900300F0222439F582E5F03400229018
:1004C00003E4E0FF75F00222F583E0FEA3E0780389
:1004D00022E0FCA3E0C39FEC9E22F074232EF58261
:1004E000E43402F583E4F022E025E02420F582E400
:1004F000341FF58322E0FEC8EDC80822902EC5E423
:10050000F0902ECDF0A3F022F582E43403F583229F
:100510009402EE648094802275F002EC122291E441
:1005200075F00122E0FCA3E0FDC3EF9DFFEE9C22ED
:10053000902EC6F0902EC57401F022902EC974281A
:10054000F09003D2E022C3EF94FEEE6480947F2209
:10055000C3EF94F6EE6480947F229DEC6480F8EE05
:1005600064809822ECF0A3EDF09003E4E022900385
:10057000E5E0FF9003E4E022900235E004F0C3944C
:100580000A22F0900227F0900301F022EEF0A3EF90
:10059000F09003C6E0229003E4EFF01212D212149E
:1005A000A8CEC313CE13D8F99003EBF0E4A3F090D8
:1005B00003E6F09003E5F09003E5E0FFC394094003
:1005C00003021761EF700302175B9003E97408F0F0
:1005D0002407A3F01212F41210FAC083C082900311
:1005E000E5E0FED082D0831210A4EE1211C61212E2
:1005F000EA9003E7F0A3EFF0121334E0601A75F00D
:1006000099EF12117AC083C0829003E5E0D082D0C6
:10061000831211C6E4F0A3F01218389003E9E0FD4C
:100620003395E0FCC3EF12153A504012137D1211BE
:100630007AC083C0829003E5E0FCD082D08312119F
:10064000C612138E121179EC1212581212B09407BE
:10065000EE6480948040030216D7C3EF94F9EE64F1
:1006600080947F40030217240216FE12183890036C
:10067000EB1212C75004A3E004F09003E9E0FF334B
:1006800095E0FEC3E49FFDE49EFC9003E71212B0E8
:1006900012153A50069003E6E004F0121479600354
:1006A000021724123B399003EA1212C7502112128A
:1006B000F41210B3C083C0829003E5E0FED082D074
:1006C000831210EB121257ECF0A3EDF00217241274
:1006D000137D12117AC083C0829003E5E0FCD082C2
:1006E000D0831211C612138E1211791212A9940A14
:1006F000EE64809480402212138512117AC083C068
:10070000829003E5E0FCD082D0831211C61213BEA2
:10071000ED1210FA1214F880281215305026121219
:10072000F412117AC083C0829003E5E0FED082D03B
:10073000831211C61213BE1210F912125774FFF56C
:10074000F01222171212F41210FAC083C082900322
:10075000E5E0FED082D0831210A41212571212EAE2
:10076000FE9003E4121215C083C0829003E5E0D02E
:1007700082D0831211C6EEF0A3EFF012136B0215B4
:1007800097121479703B9003E4E0FF242E12142C8E
:10079000E0702E742E2F12142C7401F0E49003E5F7
:1007A000F01212F41210B3C083C0829003E5E0FE91
:1007B000D082D0831210EB121257121366E0B409E4
:1007C000E09003E6E0C39404403A9003E4E0FF12B3
:1007D00039899003E4E0FF123737EF602FE490038C
:1007E000E5F01212F41210B3C083C0829003E5E06A
:1007F000FED082D0831210EB121257121366E0B4AF
:1008000009E080089003E4E0FF123ADF9003ECE097
:10081000C39404403A121334E070341239659003E3
:10082000E4E0FF1237E8EF602EE49003E5F01212E7
:10083000F41210B3C083C0829003E5E0FED082D0F2
:10084000831210EB121257121366E0B409E02290E3
:1008500003E4E0FF123AD0229003E7E0FEA3E0FFBA
:10086000123B39221227E3E49003D1F090001FE0FD
:10087000FF9003D1E0C39F4003021AD9E0FF121298
:10088000BBE4F0A3F01213A5E4F0A3F09003DF1291
:10089000145C7409F0EF7003021AD0121D17900354
:1008A000D1E0FF121576E49003D2F09003D2E0FF7E
:1008B000C394094003021A091214796006900303D5
:1008C000E06023900020E0701D900316E070179008
:1008D00003D1E075F099A42475F582E5F034001297
:1008E00011C3E4F0A3F09003D2E0FD7003021A00FC
:1008F0009003D11212DFE070289003D1E0FC1212B5
:10090000D21214A8CEC313CE13D8F9FF75F099EC08
:1009100012121975F002ED1222911214B150468094
:100920002E9003D1E0FD1213271214A8CEC313CECC
:1009300013D8F9FF75F099ED121219C083C0829097
:1009400003D2E0D082D0831211C61214B150161215
:100950001212C083C0829003D2E0D082D0831211E1
:10096000C6E4F0A3F09003D1E0FF75F0991210FAFD
:10097000C083C0829003D2E0FED082D0831211C621
:10098000E0FCA3E0FD1213A5EC8DF01222179003FA
:10099000D1E0FF12121675F002EE1210EEC083C005
:1009A000829003D2E0D082D0831211C6E0FEA3E091
:1009B0002DFFEE3CFE9003D1E0FD1212BB12138E10
:1009C000ED121219C083C0829003D2E0D082D0838E
:1009D0001211C6E0FEA3E0FFC39003E0E09FEE64C7
:1009E00080F89003DFE064809850129003D2E0FD1D
:1009F0009003DFEEF0A3EFF09003E3EDF01212129C
:100A0000C083C0829003D2E0D082D0831211C6E0AE
:100A1000FEA3E0FF9003E2E02FF09003E1E03EF060
:100A20009003D2E004F002188B9003DFE0FAA3E019
:100A3000FBC39003E2E09BF09003E1E09AF0E0FE5C
:100A4000A3E0FF7C007D071221E19003E1EEF0A31B
:100A5000EFF0C3EB9FFFEA9EFED3EF1214F040319C
:100A6000A3E06409602B1212B7C083C082E0FEA32A
:100A7000E0FF9003DF121504D082D083F0A3EFF0E3
:100A80009003E1E0FEA3E0FF1212B7EE8FF0122216
:100A9000179003D1E0FF1212BBE0FCA3E0FDEF12C0
:100AA0001203ECF0A3EDF09003D1E0FF1213A6E0E7
:100AB000FCA3E012122D12129EECF0A3EDF09003B5
:100AC000F5E0602C9003D1E0B4010F121203E0FFB7
:100AD000A3E09002EECFF0A3EFF09003D1E0B402D8
:100AE0000F121203E0FFA3E0900233CFF0A3EFF068
:100AF0009003D1E004F002184CE4900228F0221296
:100B0000304C758A30538AEF0000007F08121020A5
:100B1000E49003D2F09003D2E0FFC39409400302B3
:100B20001CF9EF902EC87013E0545FF0A3746AF0C4
:100B3000902EC374A5F0A3E4F0800EE044F0F09092
:100B40002EC374C0F0A37403F09003D2E0901F177B
:100B500093902ECAF0E49003D1F090001FE0FF9034
:100B600003D1E0FEC39F4003021CF074042E121454
:100B7000E8E0FFFDE4F5E2EDC39408503874351267
:100B80001510C083C0821214D58002C333D8FCD0A4
:100B900082D083F0902ECD7401F0C083C0821214F5
:100BA000D58002C333D8FCD082D083F0902EC0749D
:100BB000C1F0021C4574F82DFD7436121510C08367
:100BC000C0821214D58002C333D8FCD082D083F007
:100BD000902ECE7401F0C083C0821214D58002C35F
:100BE00033D8FCD082D083F0902ECB74F4F0EDB4E7
:100BF0000510902EC97420F0902EC374C0F0A37419
:100C000004F0ED6406702512151B6010902E4E3016
:100C1000E0057408F0800B7488F08006902E4E7406
:100C200004F0902EC374ADF0A37406F0ED64077069
:100C30002212151B600D902E4F30E0028008748246
:100C4000F08006902E4F7402F0902EC37457F0A3DC
:100C50007407F0EDC3940640069003D2E06006905E
:100C60002EC074C2F0EDC39406400B9003D2E07026
:100C700005CDEFCD8027E4FFFE900001742EF0A398
:100C8000E4F09003D1E024041214E8E0FDE5E22052
:100C9000E20B0FBF00010EBE07DFBFD0DC53E2FB4B
:100CA0001214DCED75F002A4FFAEF0900002E02F0C
:100CB000F0900001E03EF0ED901F5093FFEDC394E3
:100CC00008400474F82DFDEDC3940640109003D243
:100CD000E0FE7009121248E4F0A3F0802A900001AF
:100CE000E475F00212222D85F082F58312135DEF78
:100CF000121280C083C0829003D2E0D082D08312CF
:100D000011C6ECF0A3EDF09003D1E004F0021B3A21
:100D10009003D2E004F0021AF5902ECBE4F0902E6E
:100D2000C6F0758A50538AEF0000007F041210202D
:100D30009002287401F0229003E4EFF0E49003E9BC
:100D4000F09003E87409F0E49003E5F09003E5E027
:100D5000FFC394094003021F16EF7003021F0D1218
:100D600014797032121278C083C0829003E5E0FEDD
:100D7000D082D0831210A4121257121544121239C5
:100D8000C083C0829003E5E0D082D0831211C6E414
:100D9000F0A3F0021F0D9003E4E0FF75F09912102C
:100DA000B3C083C0829003E5E0FED082D0831211ED
:100DB000C6E0FCA3E0FD1212481212EAFE9003E620
:100DC000F0A3EFF0123B399003E81212C740030280
:100DD0001E939003E6E0FEA3E0FF9400EE6480948F
:100DE00080400DE024FFF09003E6E034FFF0802225
:100DF000C3EF94FFEE6480947F50109003E7E024EB
:100E000002F09003E6E03400F08007E49003E6F09F
:100E1000A3F012154E12143412114BE0B4011890C5
:100E200003E41211B512135DEE1210B31211C5ECEA
:100E3000F0A3EDF0021EE69003E6E0FEA3E0FF1251
:100E40001234C083C0829003E5E0FCD082D08312CC
:100E500011C612138EED12123C1212A91214F04098
:100E60001F121234C083C0829003E5E0FCD082D010
:100E7000831211C61213BEED1210B31214F8802D96
:100E80001215264003021EE69003E4E0FF12123919
:100E9000C083C0829003E5E0FED082D0831211C6E9
:100EA0001213BE1210B212125774FFF5F01222176D
:100EB000021EE69003E9E004F0121278C083C082BB
:100EC0009003E5E0FED082D0831210A412125712D4
:100ED0001544FF121216C083C0829003E5E0FED0D5
:100EE00082D0831211C6E0FCA3E0C3940AEC6480B4
:100EF0009480401275F099EF121437F583E5822E35
:100F00001211507401F012154EFE12143412114BCE
:100F1000E06401701812113EE00412113DE0D39418
:100F200005400A9003E5E0FF121123E4F09003E589
:100F3000E004F0021D2C223F3F3F3F3F3F3F3F3F39
:100F4000003200320064012C025800640258000490
:100F5000001E000A000A000F0064000A000C000CCA
:100F6000000000000000000000000000000101017E
:100F70000D0E0F030405060708090A0B0C000102F9
:100F800000320032003200320032003200320032D1
:100F900000320032003200320032003200320032C1
:100FA0000037003700370037003700370037003789
:100FB0000037003700370037003700370037003779
:100FC00000280028002800280028002800280028E1
:100FD00000280028002800280028002800280028D1
:100FE000002D002D002D002D002D002D002D002D99
:100FF000002D002D002D002D002D002D002D002D89
:1010000000600060006000600060006000600060E0
:1010100000600060006000600060006000600060D0
:101020000065006500650065006500650065006598
:101030000065006500650065006500650065006588
:1010400000580058005800580058005800580058E0
:1010500000580058005800580058005800580058D0
:10106000002D002D002D002D002D002D002D002D18
:10107000002D002D002D002D002D002D002D002D08
:1010800000C800C800C800C800C800C800C800C820
:1010900000C800C800C800C800C800C800C800C810
:1010A00000CD00CD00CD00CD00CD00CD00CD00CDD8
:1010B00000CD00CD00CD00CD00CD00CD00CD00CDC8
:1010C00000BE00BE00BE00BE00BE00BE00BE00BE30
:1010D00000BE00BE00BE00BE00BE00BE00BE00BE20
:1010E000002D002D002D002D002D002D002D002D98
:1010F000002D002D002D002D002D002D002D002D88
:1011000000FA00FA00FA00FA00FA00FA00FA00FA0F
:1011100000FA00FA00FA00FA00FA00FA00FA00FAFF
:10112000BB010689828A83E0225002E722BBFE02CD
:10113000E32289828A83E49322BB010CE58229F5AC
:1011400082E5833AF583E0225006E92582F8E6221B
:10115000BBFE06E92582F8E222E58229F582E583D5
:101160003AF583E49322BB010689828A83F02250F8
:1011700002F722BBFE01F322F8BB010DE58229F53F
:1011800082E5833AF583E8F0225006E92582C8F625
:1011900022BBFE05E92582C8F222EF8DF0A4A8F05B
:1011A000CF8CF0A428CE8DF0A42EFE22BC000BBE66
:1011B0000029EF8DF084FFADF022E4CCF875F00843
:1011C000EF2FFFEE33FEEC33FCEE9DEC984005FC78
:1011D000EE9DFE0FD5F0E9E4CEFD22EDF8F5F0EE40
:1011E0008420D21CFEADF075F008EF2FFFED33FD2B
:1011F0004007985006D5F0F222C398FD0FD5F0EACB
:1012000022C2D5EC30E709B2D5E4C39DFDE49CFCD5
:10121000EE30E715B2D5E4C39FFFE49EFE12218CA9
:10122000C3E49DFDE49CFC800312218C30D507C3F0
:10123000E49FFFE49EFE22C5F0F8A3E028F0C5F08D
:10124000F8E582158270021583E038F022A3F8E0F9
:10125000C5F025F0F0E582158270021583E0C838EC
:10126000F0E822EB9FF5F0EA9E42F0E99D42F0E8BB
:101270009C45F022ECF0A3EDF0A3EEF0A3EFF022FA
:10128000A8828583F0D083D082122277122277122F
:101290002277122277E473E493A3C583C5F0C58354
:1012A000C8C582C8F0A3C583C5F0C583C8C582C8B8
:1012B00022A42582F582E5F03583F58322EF4E6086
:1012C00012EF60010EEDBB010B89828A83F0A3DF70
:1012D000FCDEFA2289F05007F709DFFCA9F022BBF7
:1012E000FEFCF309DFFCA9F0229003D1747EF0E448
:1012F000A3F090001FE0FE9003D2E0FFC39E4003E6
:10130000022474123856EF600312148C9003D2E05A
:10131000FA1212E0E060030223869003D2E0FF128B
:1013200012D21212FDEF1210DFE0FEA3E0C39DEE19
:101330009C404C9003D2E09003D1F01212E0740173
:10134000F0900226E004F0900300F09003D2E0FF5A
:1013500024221213467401F0123AFD9003D2E0FFEA
:10136000123B0C9003D2E0FF1239F59003D2E0FF5C
:10137000123A3D9003D2E01213397401F08012CF7B
:10138000EACF1237ADEF60099003D2E0121339E4CF
:10139000F09003D2E0FF12388BEF700302246BE46D
:1013A0009002270224669003D2E0FF121327121244
:1013B000FDEF1210DFE0FEA3E0C39DEE9C500302A0
:1013C00024309003D2E09003D1F01234D5EF7003B3
:1013D00002246BE4FF9003D2E0FE75F0991210B383
:1013E0001211C512135DEE1210FA1211C5ECF0A322
:1013F000EDF00FEFB409DE9003D21212DFE4F090AB
:101400000020E0FF7009900316E07003022482EFD1
:101410006010900316E0600A12126F121308440560
:10142000802A900020E06010900316E0700A1212EB
:101430007012130844018014900020E0706490033F
:1014400016E0605E12126F1213084404F0C28A2282
:101450009003D2E0FF1212E0E4F0123B2A9003D294
:10146000E0FF1239D19003D2E0FF123B1B9003D270
:10147000E0FF123A199003D2E024221213467401BD
:10148000F0900227E004F0900301F09003D2E00412
:10149000F00222D29003D1E0FF90022BE06F6002B5
:1014A000EFF022CBEFCB121299E0FEA3E0FF121275
:1014B00002E0FCA3E0FDC39FEC9E5003022571E413
:1014C0002DFFEC3404FE1212991215041211A1EE34
:1014D000F0A3EFF0121299E0FEA3E0FF121202E077
:1014E000FCA3E0C39FFFEC9E1210DAEEF0A3EFF036
:1014F000121398E493FE740193FF1210DBE0FCA337
:10150000E0FDD39FEC9E4058121398E493FE7401C3
:1015100093FFC3ED9FFFEC9EC313FEEF13FF121367
:10152000987401932FFFE4933E1210DA12156C6445
:101530000360030225A8EBB4010F1210DCE0FFA347
:10154000E0900231CFF0A3EFF0EB6402707A12105A
:10155000DBE0FFA3E090032CCFF0A3EFF00225A87F
:101560001210DBE0FEA3E0FF7C007D6312217A0D08
:1015700012218C1210DB12156CB4030BEBB40107B3
:10158000E4900231F0A3F0EB6402703C90032C80F5
:1015900034121202E0FEA3E0FF1212991214B1C33A
:1015A000940475F002EB50121210DFE4F0A3F01275
:1015B00011A27404F0A3E4F0800E1210DFE4F0A393
:1015C000F01211A2E4F0A3F0EB640170441210DBFE
:1015D0001212B0949AEE940140081210BFEEF0A3DC
:1015E000EFF01210DB121453900350F0EDA3F01241
:1015F00011A21212B094DCEE94054008121186EE8E
:10160000F0A3EFF01211A2121453900354F0EDA3C3
:10161000F0EB640270441210DB1212B0949AEE9454
:101620000140081210BFEEF0A3EFF01210DB12140D
:1016300053900352F0EDA3F01211A21212B094DCF9
:10164000EE94054008121186EEF0A3EFF01211A2FD
:10165000121453900356F0EDA3F022900236E0648A
:1016600002703090030204F09003CAE0B4010890C5
:10167000033D7401F08005E490033DF0900344E0E5
:10168000B401089000007401F08005E4900000F0BF
:101690007F0222E4FE90001FE0FFEEC39F400302A2
:1016A00027E0121343E0640160030227DC741C2E60
:1016B0001212E2E0FC6003022728EE6401703D1282
:1016C0001309900301E0FD6401701B900300E0909A
:1016D0000346B40109E0440912126E048015121287
:1016E0006B1215628016ED900346B4020BE04405C0
:1016F00012126E1214BA800412126BF0EE640260C1
:10170000030227D5121309900301E0FD6401701C48
:10171000900300E0900346B40106121372E48021A6
:10172000E0440412126E1215620227D5ED900346B2
:10173000B40205E044058003E04404F0E490002096
:10174000F0900316F00227D5EC640160030227D560
:10175000EE6401704F121309900300E0FFB4020B16
:10176000900346E0440A1213758013EF640170265B
:10177000900227E0900346B4010C121372E4900328
:10178000161214BA801EE04402121375E490031678
:10179000F012148D800E900346E04402121375E49B
:1017A000900316F0EE6402704C121309900300E0EF
:1017B000B40213900346E0440AF09003167401F05B
:1017C000900020F0802F900226E06401701C9003AE
:1017D00001E0900346B40105E044098013E04408A9
:1017E00012126E04F012148C800B900346E0440831
:1017F00012126E04F0121343E4F0C28A0E02267530
:101800007F0422E49003E5F0A3F09003E97403F071
:101810002405A3F0122C87E49003E4F09003E4E0A5
:10182000FFC3940940030228F275F0021210F91266
:1018300012FF1210B21212EAFE9003E7F0A3EFF0CB
:10184000123B399003E91212C750249003E6E004DA
:10185000F0A31211581212B0940AEE6480948040E2
:101860000302289412153040030228CA0228B790B8
:1018700003E5E004F012147970709003E7E0FEA332
:10188000E0FF123B399003EAD31212C8401412143D
:101890009F1210B375F0021210F4ECF0A3EDF002F9
:1018A00028CA9003E71211581212B09464EE6480B3
:1018B000948040189003E4E0FD75F00212117A1252
:1018C0001465ED1210FAE475F001801BC3EF949CCF
:1018D000EE6480947F501312149F12117A121465D3
:1018E0001210F974FFF5F012221712149F1210FA59
:1018F0001212FF1210B21212EAFE9003E4E075F029
:1019000002121219EEF0A3EFF09003E4E004F002EB
:1019100027FC9003E5E0C3940440028031C39001AA
:1019200011E09408900110E06480948040269001BA
:10193000AAE094089001A9E0648094804016900089
:1019400078E09403900077E06480948040069002F1
:101950002D7401F09003E6E0C39406403790022D09
:10196000E06031E4FF1239ADE4FF123772EF602915
:10197000E490022DF09003EBF090001FE0FF900345
:10198000EBE0FEC39F5012121429E4F09003EBE049
:1019900004F080E5E4FF123AEE22C0E0C083C0828A
:1019A000C0D0E8C0E0E9C0E0EAC0E0EBC0E0EFC0D2
:1019B000E0D2AFE5DB30E418D2081236C430E102E1
:1019C0008034900345E5DFF09003C7E4F0022AE697
:1019D000E5DB30E5169003417401F09003CCE06044
:1019E00005E4F0022AE6C208022AE61236C430E113
:1019F0002AE5DB30E00FA31236BB1236D2122119D2
:101A0000F5DF022AE69003C8E064016003022AE6DB
:101A1000308A03022AE6D28A022AE69003CC7401B5
:101A2000F09003C7E0700DA3E5DFF09003C77401E9
:101A3000F0022AE69003C8E09032D393FFB4FF0F80
:101A4000900345E5DFF09003C8E004F0022AE0EFE0
:101A5000640F702F9003CD1236BB9003C8E0FF12C5
:101A600036F0540F1221469003CD1236BB9003C8B6
:101A7000E0FF04F01236F0FFE5DF54F04F1221468C
:101A8000022AE09003CD1236BB1236D2E5DF1221D6
:101A9000589003C8E0FF64147044E5DFB42025903B
:101AA000033EE06004E4F0800B9003CB7401F090FF
:101AB00003C6E4F09003CA7401F0900344E4F0908C
:101AC000024804F0E5DFB410159003CBE4F0900376
:101AD000C6F0900344F09003CAF0900248F0EFB4CF
:101AE000161EE5DFB4200B9003447401F09003CA86
:101AF000E4F0E5DFB41009900344E4F09003CAF089
:101B0000900343E004F075DBFFD0E0FFD0E0FBD0B2
:101B1000E0FAD0E0F9D0E0F8D0D0D082D083D0E0A5
:101B2000329003CBE060069003C6E004F09003C659
:101B3000E0B4010BE49003CBF09003C6E004F09016
:101B400003C6E0B40320D3900232E09464900231E3
:101B5000E09400500E90032DE0946490032CE094E8
:101B60000040031214809003CAE06401705890038F
:101B7000D1F01213B24003022C5CE0FF25E0248078
:101B8000F582E4341F1211CCFF25E02460F582E4D5
:101B9000341F1212251212D61211E2FF25E024A0E2
:101BA000F582E4341F12122512132B1211E2FF25C5
:101BB000E024C0F582E4341F12122512149612118B
:101BC000E204F0022B52900344E064017058900349
:101BD000D1F01213B2504CE0FF25E02480F582E4EE
:101BE00034201211CCFF25E02460F582E434201269
:101BF00012251212D61211E2FF25E024A0F582E48C
:101C0000342012122512132B1211E2FF25E024C0FA
:101C1000F582E434201212251214961211E204F017
:101C2000022BB2022C5CE49003D1F01213B2504CA0
:101C3000E0FF25E02400F582E434201211CCFF25DA
:101C4000E024E0F582E4341F1212251212D612119C
:101C5000E2FF25E02420F582E4342012122512133D
:101C60002B1211E2FF25E02440F582E43420121209
:101C7000251214961211E204F0022C0B90020CA310
:101C8000E090034AF0900347E0B4AA03123429908D
:101C90000361E07011A3E0B4100CE4900361F0A3C1
:101CA0007410F012348622E49003F0F09003EF7485
:101CB00003F0E49003ECF09003ECE0FFC3940940E0
:101CC00003022E0475F0021210B2E0FCA3E012121F
:101CD0002D1212811212EAFE9003EDF0A3EFF01222
:101CE0003B399003EF1212C74003022D969003ED8B
:101CF000E0FEA3E09400EE64809480400DE024FFB9
:101D0000F09003EDE034FFF08016C3EE6480948021
:101D1000500E9003EEE004F070069003EDE004F046
:101D200012134EE0B4013075F002EF121219E0FE0A
:101D3000A3E0C3941EEE648094804003022DD290F1
:101D400003ECE075F00212128075F0021210ADEC97
:101D5000F0A3EDF0022DD29003EDE0FEA3E0FF90A2
:101D600003ECE0FD75F00212123CEE8FF012221728
:101D700075F002ED12123C1212B01214F0401890DD
:101D800003ECE0FD75F00212123C121465ED121026
:101D9000B3E475F001801A12152650569003ECE05A
:101DA000FF75F00212123C1214651210B274FFF5A6
:101DB000F0122217803C9003F0E004F09003EC75E1
:101DC000F00212127E1212FF1210B2ECF0A3EDF02C
:101DD0009003ECE0FF75F002121219E0FCA3E0C3DF
:101DE000941EEC64809480400974B42F12135574CF
:101DF00001F09003ECE0121353E0B4011E9003ECE9
:101E0000E0FF24BD121471E00412146DE0D39405B8
:101E1000400912134EE412146DE4F09003ECE00458
:101E2000F0022C97227F05123568EF600AE49003D8
:101E30003EF07F05123AB2900236E024FE6018149C
:101E4000601E147003022EFD24036003022F75121E
:101E50001485E49002FFF09002367403F0022F76AE
:101E6000121ADF900228E07003022ED69002FFE0E3
:101E700004F0E49003D0F090001FE0FF9003D0E066
:101E8000C39F5072E4FF1211B212135DEE1210FAEA
:101E90001211C5ECF0A3EDF01211B212135DEE12A7
:101EA00010B31211C5ECF0A3EDF00FEFB409D79009
:101EB00003D0E0FF1210DCE4F0A3F0EF1211A374E2
:101EC00004F0A3E4F0EFB40110E4900350F0A3F0A9
:101ED0009003547404F0E4A3F0EFB40210E4900310
:101EE00052F0A3F09003567404F0E4A3F09003D0F2
:101EF000E004F0022E579002FFE0C3940350030267
:101F00002F75900012747EF0E4900229F09002FF89
:101F1000F07F0E123AC19002367404F0229003C68C
:101F2000E0B4020B7403F07F04123AB21238EE9060
:101F300003C6E0B403107F04123568EF60087F0425
:101F4000123AB2121480123521121ADF1235219082
:101F50000228E06040121844123521E49003D0F0CA
:101F600090001FE0FE9003D0E0FFC39E5019123690
:101F7000361236F99003D0E0FF12248312352190F7
:101F800003D0E004F080D91238C01222C912263BD7
:101F9000900236EFF0227E027F107D007B017A00F6
:101FA000792112229D123677E490023BF090033D96
:101FB000E090035970057410F080037420F09000D5
:101FC00000E090035B70057410F080037420F01241
:101FD0002B01E4FE90001FE0FFEEC39F5079E4FF69
:101FE00075F099EE12117A1211C51213BEEEA424E7
:101FF000ABF582E5F0340012114BE4F075F099EE88
:10200000A42499F582E5F034001211C3E4F0A3F0A2
:10201000121123E4F00FEF640970C5CFEECF123A2E
:10202000DF123AEE121429E4F0123AFD123B1B12B1
:102030003B0C123B2A741C2E1212E2E4F0121343E2
:10204000E4F0900225747EF0E4A3F0A3F090030086
:10205000F0A3F00E022FB4E490022DF090022B7446
:102060007EF0900012F0E490022AF0229003C9E082
:102070006013D3940A4003740AF09003C9E014F08B
:10208000E07002C208300803023103E5DB30E203EE
:10209000023103D2AF53A88053A90853AA0843A919
:1020A00008758DA0758E1C758B0843AA08E4F5860B
:1020B00020085FE5DB20E25A758A30538AEF438AB5
:1020C00084200845E5DB20E240758703000000AF6F
:1020D0008E90031AE4F0A3EFF090031AE4F0A374D7
:1020E0001CF090031AE07002A3E0601D90031BE057
:1020F00024FFF090031AE034FFF012155840E3E497
:10210000F012109612144180D9758A50538AEF004C
:102110000000758B0D758EFF758DE053AA0143AAE3
:1021200001D2AF22E49003D2F0FF9003D1F0EF147C
:10213000601E14603514604C14605B24047074904D
:1021400003D37401F0A3742FF0A37458F002318DFF
:102150001236B8900001122119FED3941F400312C9
:1021600036DF1221006E704B80431236B8900002A9
:10217000122119FED3940640031236DF1221006E9D
:10218000703180291236B8900003122119FE1221F5
:10219000006E701F80171236B8900004122119FECD
:1021A000648B60031236DF1221006E70069003D13B
:1021B000E004F00FEF6405600302310E9003D1E0FC
:1021C000B40504A37401F09003D2E0FD600790030E
:1021D0005AE0547FF0CFEDCF22758A50538AEF90AA
:1021E00003F37411F09003F27422F09003F474334B
:1021F000F075997F759A80E4FFFEC296000000207A
:10220000970ED2960000003097069003F37487F083
:102210000FBF00010EEF640A4E70DF7590FF7599D5
:102220003F759AC0E4FEFF3096032097069003F2B4
:102230007487F00FBF00010EEF640A4E70E9E4F5F9
:10224000AD75AEE075AF1DF5AC75800C7589FF7589
:10225000913E75991FF59675931CF59BF595F59232
:10226000F59AD28A9003F504F0758B0D758EFF7583
:102270008DE022023820E493A3F8E493A34003F610
:102280008001F208DFF48029E493A3F85407240CBA
:10229000C8C333C4540F4420C8834004F45680019B
:1022A00046F6DFE4800B01020408102040809033E2
:1022B00053E47E019360BCA3FF543F30E509541FF3
:1022C000FEE493A360010ECF54C025E060A840B89F
:1022D000E493A3FAE493A3F8E493A3C8C582C8CA1D
:1022E000C583CAF0A3C8C582C8CAC583CADFE9DEF0
:1022F000E780BE0F000000FFFF00000000FFFFFFAF
:10230000FFFFFFFFFFFF00000000000000000000D3
:1023100000000000000000000000000000000000BD
:1023200000000000000000000000000000000000AD
:10233000000000000000000000000000000000009D
:10234000000000000000000000000000000000008D
:10235000000000000000000000000000000000007D
:10236000000000000000000000000000000000006D
:102370000000004102FF004102350041030200411C
:102380000020004103160041033D004100000042CF
:102390000231000042032C00004102480041023B90
:1023A00000410237004103030042031A00004103C9
:1023B000C7004103C80042033F0000410341004100
:1023C00003430041034200410345104103CB004158
:1023D00003C60041033E014103CA0041034400C15A
:1023E000084103C9004103CC0000902EC0E4F090E6
:1023F0002ECB74F4F0902F58E0540F24F0902EC898
:10240000F0902ECC7448F0902EC97428F0A3743F3D
:10241000F0902E40748112128CF0A3F0A3041212DB
:102420008C7402F0A3F0902EC67434F0902EC17418
:10243000B0F0A3E4F0A37480F0A37407F043E310BA
:10244000123A7E90001FEFF0229003D27410F0A396
:10245000E4F0A3743FF0A374FFF0E4FDFCF9758A87
:1024600010538AEF0000009003D2E0FEA3E0123682
:10247000E6FF69F90DBD00010CBC2FEBBDFFE89034
:1024800003D4E0FEA3E0F5828E83E49369700890A4
:1024900003477405F08005E4900347F0758A5053B4
:1024A0008AEF000000227F007E10E4FDFC9003D242
:1024B000F0A3F0758A10538AEF000000EF1236E6A1
:1024C000FB9003D3E02BF09003D2E03400F00DBD7D
:1024D00000010CED7003EC643070E19003D2E0FC7D
:1024E000A3E0FDEC900361F0EDA3F0758A50538AF0
:1024F000EF000000229003D3EFF0E0FF2417121446
:1025000021E0603A900248E064017011EF12107E01
:1025100012125E901F26121115402380129003D3D1
:10252000E012107E12125E901F2C121115400F90B7
:1025300003D3E02417F582E43403121318227F003A
:1025400022900237E024FE601114602524037037C6
:102550003088349002377402F02220882A900237A3
:102560007403F09003037401F07F0E123AC1023934
:10257000167F0E1235AEEF600E7F0E123AC1E49058
:102580000237F0900303F0229003D1EFF0C3940FD1
:102590005039E0FF24971213C9E0602FEF25E025A2
:1025A000E024B2F582E4340212108912125E900324
:1025B000D11214C8121115400F9003D1E02497F5E1
:1025C00082E43402121318227F00227F002290033B
:1025D000D1EFF0C3940F5039E0FF24491213D4E037
:1025E000602FEF25E025E0245BF582E43402121031
:1025F0008912125E9003D11214C8121115400F9067
:1026000003D1E02449F582E43402121318227F003A
:10261000227F0022C0E0C0F0C083C082C0D0E8C0EA
:10262000E0ECC0E0EDC0E0EEC0E0EFC0E0D2AF1201
:1026300015584008E4F0121096121441D0E0FFD073
:10264000E0FED0E0FDD0E0FCD0E0F8D0D0D082D0E9
:1026500083D0F0D0E032CBEFCBE49003D112145C06
:10266000F0A3F0EB640170121211EEE0900396F00B
:10267000121202A3E09003978015EB640270171208
:1026800011EEE090039AF0121202A3E090039BF087
:10269000ECA3F0EDA3F0227E007F807D007B017A29
:1026A00003794612229D9003467405F0A3F0E4A33B
:1026B000F090035874ABF090035A74A8F09003F3B1
:1026C000E090034CF09003F2E090034DF09003F49F
:1026D000E090034EF00231049003D3E0FBA3E0FA54
:1026E000A3E0F9229003C9740AF09003CCE4F0E56A
:1026F000DB229003C8E0FF04F08F827583002290F4
:1027000003D27401F0222DF582EE3CF583E493228E
:10271000E92FF9E43AFA0221009003F5E06037C3AB
:102720009002EFE094E09002EEE0942E50069003C9
:10273000F47487F0C3900234E09428900233E0945C
:102740002350069003F47487F0E49003F5F09003AF
:10275000F4E090034EF0229003EDEFF0E0FF242E22
:102760001213EAE06029EF25E025E02431F582E448
:10277000340312108912125E901F32121115400F8D
:102780009003EDE0242EF582E43403121318227F27
:1027900000229003ECEFF0E0FF24071213F5E06055
:1027A00029EF25E025E0240AF582E434031210899C
:1027B00012125E901F34121115400F9003ECE024AA
:1027C00007F582E43403121318227F00229003D30A
:1027D000EFF0E0FF2438121400E06029EF25E02537
:1027E000E0243CF582E4340212108912125E901F3C
:1027F00022121115400F9003D3E02438F582E434FF
:1028000002121318227F00229003EDEFF0E0FF2464
:10281000F01213DFE06026EF25E025E024F3F582D7
:10282000E43402121089901F24121109400F900302
:10283000EDE024F0F582E43402121318227F002226
:1028400075200153A87F1231B912393E43A8801276
:10285000104E121066123A61EF24E0600A241070E4
:102860000AC283C2828004D283D282122B01758D68
:10287000E0122E0580DF9003D3EFF0E0FF24031277
:10288000140BE06023EF25E025E02406F582E43414
:1028900000121089121106400F9003D3E02403F5B3
:1028A00082E43400121318227F00229003D3EFF049
:1028B000E0FF2458121416E06023EF25E025E02401
:1028C000A6F582E43402121089121106400F90031B
:1028D000D3E02458F582E43402121318227F002238
:1028E000E4FFFE90001FE0FDEEC39D501BEF1210B1
:1028F000DC1212FFEE1210DFE0FAA3E0D39DEA9C97
:102900004003CFEECF0E80DB90022CEFF022CBEF16
:10291000CBEBD3940F501E1213C6E070181213C6DF
:102920007401F012109612131124B2F582E43402ED
:10293000F58312225422CBEFCBEBD3940F501E120F
:1029400013D1E070181213D17401F0121096121303
:1029500011245BF582E43402F583122254229003A1
:10296000CD7401F0A37403F0A37446F0E4F5DA75B6
:10297000DA4043DA2075D74075DA5843A90875B8AC
:102980000875F8082212131F501E1213DCE070188D
:102990001213DC7401F012109612131124F3F58255
:1029A000E43402F5831222542212131F501E121314
:1029B000E7E070181213E77401F012109612131169
:1029C0002431F582E43403F5831222542212131FBA
:1029D000501E1213F2E070181213F27401F012106C
:1029E00096121311240AF582E43403F5831222545B
:1029F0002212131F501E1213FDE070181213FD74E3
:102A000001F0121096121311243CF582E43402F501
:102A1000831222542212131F501E121408E0701841
:102A20001214087401F01210961213112406F58284
:102A3000E43400F5831222542212131F501E121484
:102A400013E070181214137401F01210961213117F
:102A500024A6F582E43402F5831222542212131FB5
:102A6000501E12141EE0701812141E7401F0121081
:102A700096121311241CF582E43403F583122254B8
:102A800022E4FD900341E06011900346E0FE54F023
:102A9000FDEE540FF0E4900341F0CFEDCF2212147D
:102AA000DCFFFEEE901F4093600974042F1214E8BF
:102AB000EEF00F0EEEB410EB22900328122260000D
:102AC0000000007E007F0F7D007B017A02794902C1
:102AD000229DEFD3940F500874972F1213C9E4F07E
:102AE00022EFD3940F500874492F1213D4E4F0222C
:102AF000EFD39403500874F02F1213DFE4F022EFA9
:102B0000D394035008742E2F1213EAE4F022EFD36B
:102B10009403500874072F1213F5E4F022EFD394B6
:102B200003500874382F121400E4F022EFD39403FA
:102B3000500874032F12140BE4F022EFD3940350C7
:102B40000874582F121416E4F022EFD3940350089F
:102B500074172F121421E4F022EE30E707C3E49F2C
:102B6000FFE49EFE220000000000000000000000C4
:102B70000000000000000000000000000000000055
:102B80000000000000000000000000000000000045
:102B90000000000000000000000000000000000035
:102BA0000000000000000000000000000000000025
:10301000000000000000000000000000000000C9E7
:00000001FF
